:100000000C943E040C9485040C9485040C94850493
:100010000C9485040C9485040C9485040C9485043C
:100020000C9485040C9485040C942C2A0C94FE2AC0
:100030000C9470200C9485040C9485040C94850415
:100040000C9485040C9485040C9485040C9485040C
:100050000C9485040C94D8200C9485040C9485048D
:100060000C9485040C9485040C9485040C948504EC
:100070000C9485040C9485040C9485040C948504DC
:100080000C9485040C9485040C9485040C948504CC
:100090000C9485040C9485040C9485040C948504BC
:1000A0000C9485040C9485040C948504A606AB0678
:1000B000B506A906AE06B306B106410743074E07CB
:1000C0004507470749074B074D0750075207540795
:1000D0005F07560758075A075C075E0761072D162A
:1000E0002D16671667169C16BC1629186518FE167D
:1000F0006518AE17AE172118651865186018BB177C
:10010000BB17BB17BB17BB17BB17BB17BB17BB175F
:10011000BB17BB17BB17BB17BB17BB17BB17CD173D
:10012000DA17E117E817F217F018F0180219021998
:10013000F918021902190219F018F018FE1802191C
:100140000219FE186B2B8D2B7B2C8D2B7B2CD22B2D
:10015000F52B7B2C4A2C5D2C6572676F646F782FB2
:100160006572676F646F785F657A5F393130646597
:10017000666536326366313637346436376430202C
:100180004020302E352E3438006572676F646F78EA
:100190002F6572676F646F785F657A5F393130649D
:1001A00065666536326366313637346436376430B7
:1001B000204020302E352E3438000000F0A100679A
:1001C00001542900C65CE00000001E001400040079
:1001D0001D0035644D001F001A0016001B0034007E
:1001E0002B00200008000700060050002C00210012
:1001F0001500090019004F004A00220017000A00EC
:1002000005000000E2002D00E00000000068000092
:1002100065002E0029000000007800004C0023003B
:100220001C000B0011000000E600240018000D0067
:10023000100052004B0025000C000E00360051004B
:100240002800260012000F0037002F002A00270088
:1002500013003342380030744E00006F3100340018
:10026000C75C0071000000300100010001000100C6
:1002700000003A001E0220022202010001003B00A1
:100280001F022102230201002B003C002F02260244
:100290002F0001002A003D0030022702300001003B
:1002A00001003E003102350035020000010001006E
:1002B0000100000001000000010001000100000039
:1002C0000100000001003F00520051002402000024
:1002D00001004000240021001E0001000100410037
:1002E000250022001F0037002800420026002300BE
:1002F000200027002A00430025022E0231002E0094
:10030000010044004500010001000100000001005F
:1003100001000100010001000000010001000100D6
:1003200001000100F60001000100F20001000100DF
:10033000F5000100F000F10001000100F4000100EF
:100340000100F300010001000100010001000100B3
:100350000100000001000100010000000100000098
:100360000100010001000000010000000100010087
:100370000100010001000000010001000100FD007A
:10038000A800A900010001000100FE00AC00AA00C5
:10039000010001000100FF00AB00AE000100010000
:1003A000010001000100AD00010001000100010099
:1003B00001000100000000000000000000002A2BE6
:1003C0002800000000000000000000000000000005
:1003D0000029000000002C1E34202122243426276E
:1003E000252E362D3738271E1F202122232425268F
:1003F0003333362E37381F0405060708090A0B0C5D
:100400000D0E0F101112131415161718191A1B1CA4
:100410001D2F3130232D350405060708090A0B0C62
:100420000D0E0F101112131415161718191A1B1C84
:100430001D2F3130354C000000000000000000008E
:1004400000000000000000000000000000000000AC
:100450000000000000000001010101010100010194
:10046000010100000000000000000000000000008A
:10047000010001000101010101010101010101016E
:10048000010101010101010101010101010101015C
:100490000100000001010000000000000000000059
:1004A000000000000000000000000000000000004C
:1004B0000001010101006801F000B40078005A0059
:1004C000643214643214783C1E1E140A05000000C5
:1004D000000101010202030405050607090A0B0CCD
:1004E0000E0F1112141517191B1D1F212325282A61
:1004F0002C2F313436393B3E414346494C4F5255FF
:10050000585A5D6164676A6D707376797C7F838603
:10051000898C8F9295989B9EA2A5A7AAADB0B3B6E1
:10052000B9BCBEC1C4C6C9CBCED0D3D5D7DADCDE08
:10053000E0E2E4E6E8EAEBEDEEF0F1F3F4F5F6F8EC
:10054000F9FAFAFBFCFDFDFEFEFEFFFFFFFFFFFFD9
:10055000FFFEFEFEFDFDFCFBFAFAF9F8F6F5F4F3FA
:10056000F1F0EEEDEBEAE8E6E4E2E0DEDCDAD7D546
:10057000D3D0CECBC9C6C4C1BEBCB9B6B3B0ADAA88
:10058000A7A5A29E9B9895928F8C898683807C7963
:100590007673706D6A6764615D5A5855524F4C4965
:1005A0004643413E3B393634312F2C2A282523211E
:1005B0001F1D1B1917151412110F0E0C0B0A09071A
:1005C000060505040302020101010000000000000D
:1005D0000000010101010101010101020202020208
:1005E00002020202030303030303030304040404DB
:1005F00004040505050505060606060607070707A0
:10060000080808080909090A0A0A0A0B0B0B0C0C4E
:100610000C0D0D0D0E0E0F0F0F10101111111212E7
:1006200013131414151516161717181819191A1A62
:100630001B1C1C1D1D1E1F1F2020212222232425C0
:100640002526272728292A2B2B2C2D2E2F2F3031FA
:100650003233343536363738393A3B3C3D3E3F400D
:1006600041424344464748494A4B4C4D4F505152F2
:1006700053555657585A5B5C5E5F606263646667A9
:10068000696A6C6D6E707173747678797B7C7E802C
:1006900081838486888A8B8D8F91929496989A9B79
:1006A0009D9FA1A3A5A7A9ABADAFB1B3B5B7B9BB8A
:1006B000BDBFC1C4C6C8CACCCFD1D3D6D8DADCDF5F
:1006C000E1E4E6E8EBEDF0F2F5F7FAFCFF1603459E
:1006D00000720067006F0044006F00780020004542
:1006E000005A00000016034500720067006F0044C6
:1006F000006F007800200045005A00000004030944
:100700000409026D00040100A0FA090400000103BD
:1007100001010009211101000122400007058103A8
:1007200008000A0904010001030102000921110166
:100730000001224D000705820308000A0904020097
:100740000103000000092111010001223600070504
:10075000830308000A0904030001030000000921C3
:100760001101000122390007058403200001120154
:10077000100100000008EDFE071301000102000156
:1007800005010906A101050719E029E71500250162
:10079000950875018102050819012905950575015E
:1007A00091029501750391010507190029F71500BC
:1007B000250195F875018102C005010980A1018517
:1007C000021601002603001A81002A830075109585
:1007D000018100C0050C0901A10185031601002655
:1007E0009C021A01002A9C02751095018100C00527
:1007F000010902A1010901A1000509190129051535
:10080000002501950575018102950175038101059A
:1008100001093009311581257F9502750881060986
:10082000381581257F950175088106050C0A380267
:100830001581257F950175088106C0C0050109064F
:10084000A101050719E029E71500250195087501A3
:100850008102950175088101050819012905950591
:10086000750191029501750391010507190029FF92
:10087000150026FF00950675088100C011241FBED3
:10088000CFEFDAE0DEBFCDBF04B603FE27C0809114
:10089000B7039091B803A091B903B091BA03873020
:1008A000904BA740B04BD1F41092B7031092B8030D
:1008B0001092B9031092BA0314BE84B7877F84BF25
:1008C0000FB6F894A89580916000886180936000CD
:1008D000109260000FBEE0E0FFE3099511E0A0E098
:1008E000B1E0E0EBFCE502C005900D92AA3DB10736
:1008F000D9F723E0AAEDB1E001C01D92A73BB207F2
:10090000E1F70E9459270C94562E0C940000109287
:10091000B9008AE08093B800089594EA9093BC00EF
:100920009091BC0097FFFCCF9091B900987F9830D0
:1009300021F0903111F081E008958093BB0084E8AC
:100940008093BC008091BC0087FFFCCF8091B900F0
:10095000887F883111F0803471F780E0089584E950
:100960008093BC008091BC0084FDFCCF08958093EF
:10097000BB0084E88093BC008091BC0087FFFCCF63
:100980009091B900987F81E0983209F480E0089551
:1009900084E88093BC008091BC0087FFFCCF8091ED
:1009A000BB00089580B38C7080BB81B3836F81BB23
:1009B000089580910001811115C080E40E948D048A
:1009C0008093000181110CC082E10E94B7048093E2
:1009D0000001811105C08FEF0E94B70480930001D0
:1009E0000E94AF0484B1807F84B985B1807F85B9CE
:1009F0008AB1837F8AB98BB1837F8BB93E98469841
:100A0000089508950C948A060E948B0B8093000130
:100A10000E94D9040E94D2042BED31E0EFE2F2E013
:100A20004EE04E0F119280E090E0D901A80FB91F5F
:100A30001C92019686309105C1F72A5F3F4F4E13F5
:100A4000F1CF0C9491080E948B0B809300010E94BF
:100A5000D9040E94D204EFE2F2E08EE08E0F1192F0
:100A60008E13FDCF089526E0829FC0011124FC0162
:100A7000E552FE4F20E030E080E041E050E0908120
:100A8000992319F09150908307C0BA01022E01C03A
:100A9000660F0A94EAF7862B2F5F3F4F3196263078
:100AA000310569F7089596E0699FB001112420E0AF
:100AB00030E090E04FE0FC01022E02C0F595E79592
:100AC0000A94E2F7E0FF06C0F901E60FF71FE552CE
:100AD000FE4F40832F5F3F4F2630310561F7089569
:100AE000AF92BF92CF92DF92EF92FF920F931F933C
:100AF000CF93DF9380910001882379F08091DA0110
:100B00008F5F8093DA01811108C00E948B0B809364
:100B10000001811102C00E941D0B8FE2E82E82E0CD
:100B2000F82E00E010E0CC24C394D12CAA24A39486
:100B3000C02F0730110500F58091000181113CC0E4
:100B400080E40E948D0480930001811112C082E133
:100B50000E94B7048093000181110BC0C601002ED2
:100B600001C0880F0A94EAF780950E94B704809329
:100B700000010E94AF0420C00A30A1F028F4083020
:100B800059F0093061F005C00C3089F070F00D307B
:100B900089F0209A289810C0219A29980DC0229A8D
:100BA0002A980AC0239A2B9807C0529A01C0539AD8
:100BB0005B9802C03E9A469880EA8A95F1F78C2F9E
:100BC0000E943305D82F0730110518F580910001D8
:100BD000811144C080E40E948D0480930001882329
:100BE00011F0B12C12C083E10E94B7048093000180
:100BF0008111F7CF81E40E948D048093000181115F
:100C0000F0CF0E94C804B82EB0940E94AF049B2D70
:100C100026C08FB181708A25799902C092E001C007
:100C200090E0892B7C9902C094E001C090E0982B61
:100C30007D9902C038E001C030E0932B7E9902C05C
:100C400020E101C020E0922B2FB12095221F222706
:100C5000221F2295220F207E922B01C090E0F701E7
:100C600080819D23D095D823D92B6C2F8D270E946E
:100C70005305F701D1937F010E94D9040F5F1F4FE5
:100C80000E30110509F054CF0E94930881E0DF91E6
:100C9000CF911F910F91FF90EF90DF90CF90BF9079
:100CA000AF900895E82FF0E0E15DFD4F8081089559
:100CB0000895611108C0FC018281882321F089E830
:100CC00091E00E94660880E090E00895FB018E3C70
:100CD0002CE5920769F08F3C2CE5920789F08D3C5A
:100CE0009C45B1F482818823A1F00E94EC1F0EC0C4
:100CF0008281882371F088E591E00E94660806C031
:100D00008281882331F081E00E94EC0F80E0089519
:100D100081E008956091FF027091000380910103CA
:100D2000909102030E949C1F56985E9825982D98DA
:100D300026982E9827982F9890E0FC013197E7305D
:100D4000F105A8F4EA5AFF4F0C94082E259A2D9A23
:100D50000895259A2D9A269A2E9A0895259A2D9AC5
:100D600004C0259A2D9A269A2E9A279A2F9A08958A
:100D700081E008950C9466060E94DE182FEF84E34C
:100D80009CE0215080409040E1F700C000000C94AE
:100D9000FE20FF920F931F93CF93DF938C01FC01F2
:100DA000C081D18180918E02811113C082818823FC
:100DB00049F0CE010E94FF1DF82E682FCE010E943F
:100DC000A21D04C0CE010E94D21DF82EBE018F2D9F
:100DD00004C0CE010E94FF1DBE010E94A808EC01C4
:100DE000B8010E94BA06882309F469C1B801CE018E
:100DF0000E94CE0A882309F462C1B801CE010E9484
:100E0000DA0B882309F45BC1C13CFCE5DF0741F440
:100E1000F8018281882309F452C10E94740F4FC1E6
:100E2000C23C8CE5D80708F0A6C0C5319CE5D907BF
:100E300008F07EC0C230ECE5DE0708F452C0F801CD
:100E40008281882309F459C00E940D20811102C0BB
:100E50000E94EC1F0E94202090E09093A9038093B1
:100E6000A803FE01E350FC45E231F10530F4E35AFA
:100E7000FF4F8091A8030C94082E8091A8038160F5
:100E800027C0826025C0846023C0806121C0806249
:100E90001FC080641DC080681BC08460886018C04B
:100EA0008E7F16C08D7F14C08B7F12C08F7E10C0C6
:100EB0008F7D0EC08F7B0CC08F770AC08B7F877FA2
:100EC00007C087FB222720F991E0922790FB87F942
:100ED0008093A8038091A8030E9424200E94DE181A
:100EE000EEC0C115FCE5DF0781F0C130DC45A9F09B
:100EF00081E08093410280934202C801DF91CF914B
:100F00001F910F91FF900C94B806F80182818823FD
:100F100009F4D5C00E94BC06D2C0F80182818823A2
:100F200009F4CDC080912C03816080932C03C7C04D
:100F3000CF3B9CE5D90741F4F8018281882309F46D
:100F4000BEC00E946710BBC0C03CECE5DE0740F0AD
:100F5000F8018281882309F4B2C00E945C0FAFC0FF
:100F6000CE3BDC4529F6F8018281882309F4A7C02D
:100F70000E947110A4C0C53C8CE5D80741F4F8016B
:100F80008281882309F49BC00E94D20F98C0C63C7E
:100F90009CE5D907D8F4F8018281C33CFCE5DF0762
:100FA00031F4882309F48BC00E94A50F88C0C43C8B
:100FB000DC4530F4882309F482C00E94930F7FC07F
:100FC000882309F47CC00E94B70F79C0C73CECE5C8
:100FD000DE0781F5F8018281882361F010924202D8
:100FE0000E94A2209093400280933F0280E20E94E0
:100FF000E21565C00E94231F81FF05C081E0809338
:101000004102809342028091420281110FC080917F
:101010003F02909140020E94AE20883C910530F43E
:1010200087E20E94C01487E20E94931580E20E942A
:10103000E91545C0C73CFCE5DF0760F5F801828192
:10104000882351F0109241020E94A22090933E0208
:1010500080933D0282E0CBCF0E94231F85FF05C015
:1010600081E080934102809342028091410281118C
:101070000FC080913D0290913E020E94AE20883CBC
:10108000910530F486E20E94C01486E20E94931516
:1010900082E0CDCFCA3C8CE5D80731F4F8018281DB
:1010A000882369F080E009C0CB3CDC4509F020CF03
:1010B000F8018281882319F082E00E94EF2780E006
:1010C000DF91CF911F910F91FF9008950F931F9380
:1010D000CF938C01F80124912223F9F030E0F9013B
:1010E000EA54FC4FC491F901EA5CFB4F249122239E
:1010F00059F081EE0E94C0148C2F0E94C0148C2FD6
:101100000E94931581EE04C08C2F0E94C0148C2F76
:101110000E9493150F5F1F4FDDCFCF911F910F914D
:1011200008950C94750B0C940205282F882339F030
:1011300090E02A3010F44D9608950697089587E2BE
:1011400090E0089508950C94A2080C94A3080895C3
:1011500096E0799FF001112494E5899FE00DF11D3F
:101160001124E60FF11DEE0FFF1FE254FE4F859193
:1011700094910895880F991FFC01E654FE4F8591C4
:10118000949108950E94A8080E94500A811520E4B5
:101190009207B0F5811540E3940708F0DBC0803E6C
:1011A0009105D8F4803C910508F069C0883A910512
:1011B00078F4853A910508F065C08130910509F40D
:1011C0006EC108F425C18430910508F068C120C1C2
:1011D0008D3B910508F461C01BC18F3F910509F05B
:1011E00048F4803F910508F0AFC0883E910508F4AF
:1011F00056C10EC1811560E2960708F0A7C0089598
:10120000811574E59707D8F4811523E5920708F056
:10121000DDC0811541E5940740F4811560E596072E
:1012200008F0A2C09F70906A0895811572E5970733
:1012300008F0B6C0982F8827816F906A08958115AD
:1012400026E5920750F4811545E5940708F0D4C0CF
:10125000982F8827846F906A0895811568E596070E
:1012600008F4D6C0811579E5970708F4CAC09C0137
:1012700030562115304208F0CBC09F71C7C0805C4A
:10128000910965C0853A910509F4C5C0863A910572
:1012900009F0C4C082E890E40895883A910509F401
:1012A000C0C0893A910509F4BFC08A3A910509F492
:1012B000BEC08B3A910509F4BDC08C3A910509F482
:1012C000BCC08B3B910509F4BBC08C3B910509F474
:1012D000BAC08D3A910509F4B9C0803B910509F473
:1012E000B8C08E3A910509F4B7C08F3A910509F458
:1012F000B6C0813B910509F4B5C0823B910509F464
:10130000B4C0833B910509F4B3C0843B910509F453
:10131000B2C0853B910509F4B1C0863B910509F443
:10132000B0C0873B910509F4AFC0883B910509F433
:10133000AEC0893B910509F4ADC08A3B910509F423
:10134000ACC080E094E40895906508959F700E9479
:10135000BA0808959C01332793FF03C0C901986C14
:101360000895C901906C0895482F437021E030E042
:1013700002C0220F331F4A95E2F73C68AC0164E0DB
:10138000569547956A95E1F74370342B8F70869593
:10139000869560E2869FC0011124822B932B0895CD
:1013A000482F4695469570E2479FA001112483700F
:1013B000992721E030E0B90102C0660F771F8A95B6
:1013C000E2F7CB01842B952B9C680895482F469516
:1013D000469570E2479FA00111248370992721E070
:1013E00030E0B90102C0660F771F8A95E2F7CB01A2
:1013F000842B952B9A6808958F719927982F8827A9
:1014000005C0982F8827806F906A0895906208958C
:1014100080E090E0089581E890E4089583E890E406
:10142000089582EE94E4089589EE94E408958AEE96
:1014300094E4089585EB94E4089586EB94E408958C
:1014400083EB94E4089584EB94E4089587EB94E4AB
:1014500008958CEC94E408958DEC94E4089583E869
:1014600095E408958AE895E4089582E995E408955D
:1014700084E995E4089581E296E4089583E296E490
:10148000089584E296E4089585E296E4089586E25C
:1014900096E4089587E296E408958AE296E4089532
:1014A0008238910549F1B0F48133910509F458C0AF
:1014B00048F48932910509F44EC08A32910509F445
:1014C00054C008958533910509F440C089339105CE
:1014D00099F00895833E910529F138F4803E9105F5
:1014E00091F0823E9105A1F00895863E9105F9F0B4
:1014F000873E910531F108952091A80320FD3AC05F
:1015000021FD38C008958091A80380FD35C032C008
:101510008091A80382FF32C08091A80384FD30C06F
:1015200083EE39C08091A80382FD28C0F5CF809159
:10153000A80383FF27C08091A80384FD21C087EE04
:101540002AC08091A80383FD1DC0F5CF8091A80318
:1015500085FD1AC01BC08091A80385FD17C014C06B
:101560008091A80386FD14C015C08091A80386FD54
:1015700011C00EC080EE0FC089E30DC082EE0BC01B
:1015800080E009C086EE07C089E205C085E303C09C
:101590008AE201C081E390E0089508950F931F93BC
:1015A000CF93FB012281211102C0C1E041C08C0117
:1015B000C0915002C11125C085319C45B1F70E94F0
:1015C000CD0A81E0809350020E94A22090934F02A6
:1015D00080934E02109243021092450210924402F0
:1015E000109247021092460210924902109248024D
:1015F00010924B0210924A0210924D0210924C022D
:1016000017C080914E0290914F020E94AE20883CFC
:10161000910558F690914302E92FF0E0EE0FFF1F7D
:10162000EC5BFD4F118300839F5F90934302C0E00A
:101630008C2FCF911F910F91089556985E98259801
:101640002D9826982E9827982F988FEF90E09093BA
:1016500089008093880090938B0080938A009093F8
:101660008D0080938C00259A2D9A2FEF80E792E0D1
:10167000215080409040E1F700C00000269A2E9A49
:101680002FEF80E792E0215080409040E1F700C0CA
:101690000000279A2F9A2FEF80E792E02150804098
:1016A0009040E1F700C0000025982D982FEF80E7CB
:1016B00092E0215080409040E1F700C00000269861
:1016C0002E982FEF80E792E0215080409040E1F784
:1016D00000C0000027982F9856985E9825982D985E
:1016E00026982E9827982F98089589EA809380004D
:1016F00089E08093810024982C983F988AB18F7C50
:101700008AB96E98479A8BB180638BB9769A0E949A
:101710001D0B0C94010580E2809300018091510221
:1017200081110EC00E94870481E0809351022FEF47
:1017300083ED90E3215080409040E1F700C000002D
:1017400080E40E948D048093000181112EC00E94CC
:10175000B70480930001811128C00E94B7048093D0
:101760000001811122C08FE30E94B7048093000121
:1017700081111BC00E94AF0480E40E948D048093FD
:101780000001811112C08CE00E94B7048093000117
:1017900081110BC00E94B70480930001811105C024
:1017A0008FE30E94B704809300010E94AF048091F0
:1017B00000010895CF93DF93813020E89207D0F0A5
:1017C000FB0122812223B1F0EC01809152028111B0
:1017D00009C08CE090E00E940E2E0E94FE0B81E07A
:1017E000809352020E94050CCE019F770E94C30C89
:1017F0000E947B0C81E0DF91CF910895809353028A
:10180000682F8CE090E00C94222EE0910201F09180
:101810000301808180935D0381FF03C081EE0E94FC
:10182000931580915D0385FF03C085EE0E9493159B
:1018300080915D0380FF03C080EE0E94931580912C
:101840005D0384FF03C084EE0E94931580915D03C5
:1018500082FF03C082EE0E94931580915D0386FF94
:1018600003C086EE0E94931580915D0383FF03C041
:1018700083EE0E94931580915D0387FF03C087EE7E
:101880000E949315809153028130A1F078F082304C
:1018900011F1843049F586EE0E94C01486EE0E9454
:1018A000931588E10E94C01488E11CC082EE0E945A
:1018B000C0141AC080EE0E94C01481EE0E94C014B1
:1018C00088E10E94C01488E10E94931581EE0E9475
:1018D000931580EE07C082EE0E94C01487E50E9437
:1018E000C01487E50E9493158FE39CE90197F1F7F7
:1018F00000C00000089580915302813029F010F05B
:10190000823041F482EE04C08CE20E94C0148CE26A
:101910000E94931580915D0381FF03C081EE0E94B8
:10192000C01480915D0385FF03C085EE0E94C01442
:1019300080915D0380FF03C080EE0E94C0148091FF
:101940005D0384FF03C084EE0E94C01480915D0398
:1019500082FF03C082EE0E94C01480915D0386FF67
:1019600003C086EE0E94C01480915D0383FF03C014
:1019700083EE0E94C01480915D0387FF03C087EE51
:101980000C94C0140895EF92FF921F93CF93DF93AE
:101990007C01CCE0D0E097010C2E02C03695279553
:1019A0000A94E2F7122F1F70812F0E9495080E945F
:1019B000C014812F0E9495080E9493152497CC3F54
:1019C0008FEFD80741F7DF91CF911F91FF90EF90F4
:1019D0000895882319F05198599A02C0519A59983C
:1019E0005098589A95E09A95F1F70000509A5898B7
:1019F00095E09A95F1F70000882311F0519A5998D3
:101A000085E08A95F1F7000008958BB18C7F8BB942
:101A10005098589A5198599A85E08A95F1F70000A4
:101A200008958AB18C7F8AB985E08A95F1F7000024
:101A3000519A599885E08A95F1F70000509A589884
:101A400085E08A95F1F7000008955098589A85E04E
:101A50008A95F1F700005198599A85E08A95F1F737
:101A600000000895CF93DF93D82FC8E08D2F8078A2
:101A70000E94E90CDD0FC150C9F780E00E94E90C1B
:101A800085E08A95F1F7000085E08A95F1F700007E
:101A900080E0DF91CF9108952BB1342F309523232F
:101AA0003BB1432B3FB7F894FC01680F791FE61751
:101AB000F70789F0819198E04BB9000000C087FFDB
:101AC0002BB9880F000000C000C000C02BB900C0B7
:101AD0009A9591F7ECCF3FBF0895AF92BF92CF9206
:101AE000DF92EF92FF920F931F93CF93DF938C01BE
:101AF000EB01CFB6D090BC00F8948091BC008B7FF6
:101B00008093BC000E94050D0E94110D84E80E9484
:101B1000320DCC0FDD1FCC0FDD1F78015801AC0E4C
:101B2000BD1EEA14FB0431F0F70181917F010E9490
:101B3000320DF7CF0E94250DCFBED092BC00579A30
:101B400040E8BE01C801DF91CF911F910F91FF9036
:101B5000EF90DF90CF90BF90AF900C944C0DEF9230
:101B6000FF920F931F93CF93DF93E901662309F44C
:101B70004BC0242F30E0EFEFF0E0E61BF109B90194
:101B8000E69F9001E79F300DF69F300D1124232F23
:101B90008B01031B11095CE3E52EF12CB7010E94B8
:101BA000E02DFB01BC01069FC001079F900D169F11
:101BB000900D1124B7010E94E02DE230F105B1F043
:101BC00040F4309779F0319711F5832F242F461B7D
:101BD00021C0E430F105A1F068F03597C1F4842FFD
:101BE000861B18C0832F262F230F14C0862F830F28
:101BF000E42F03C0E42FE61B842F432F2E2F0AC0AF
:101C0000842F462F430F06C0842F242F03C080E06B
:101C100020E040E0E42FF0E0E353FA4F4491E22F5C
:101C2000F0E0E353FA4F9491E82FF0E0E353FA4FDA
:101C3000E49149839883EA83DF91CF911F910F91BB
:101C4000FF90EF90089588E090E00C94162EAB0181
:101C5000BC0188E090E00C94342EEEE5F3E083E0E4
:101C6000808310925F038FEF8283838360915E0392
:101C700070915F0380916003909161030C94270E33
:101C800080915E0380FF06C06FE070E086E693E01F
:101C90000C946D0D80E090E0FC01EA59FC4F11823C
:101CA0001082128204968C339105B1F7EDCF20E0BB
:101CB00030E0F901EA59FC4F8183608342832C5F55
:101CC0003F4F2C333105A9F70C94400EEF92FF9251
:101CD0000F931F93CF93DF9300D000D0CDB7DEB723
:101CE00000915E0310915F032091600330916103C6
:101CF000009362031093630320936403309365039E
:101D000020915E0320FF21C0042FF62EE92E182F0C
:101D10009E012F5F3F4F0E94AF0D8091620310FB29
:101D200087F9809362031695809163038078182B5E
:101D3000E0FA17F910936303F092640300936503CC
:101D40004B8169818A810E94570E0F900F900F90EE
:101D50000F90DF91CF911F910F91FF90EF90089519
:101D60008F929F92AF92BF92CF92DF92EF92FF92AB
:101D70000F931F93CF93DF93EC01062F142F8091C5
:101D80005E0380FF8CC0982F9E77923021F4CE01A5
:101D90000E94660E5AC0E82FE695EF739EE39E0FF1
:101DA0009F73943018F4109161034FC09AE39E0F13
:101DB0009F73993070F4881F8827881F90915F0364
:101DC000292F220FC22FC82B97FB992790F9D92FC3
:101DD0003CC087E28E0F8F738A30B8F5F0E07997B8
:101DE000E0FD02C021E001C02FEFEE7FEA54FB4F7F
:101DF000859194916FE070E00E94E02D26036001D0
:101E0000279FD00C11244E0188E9881A8EEF980A7A
:101E100086E6E82E83E0F82E98E6A92EBB24B3943C
:101E2000C401B5010E94E02D9701412F602F0E944F
:101E3000AF0D8C0C9D1C94E0E90EF11C82EAE816B3
:101E400083E0F80669F70E94400E80915E039C2FA4
:101E5000C0FB87F980935E03969580915F0380783D
:101E6000892BD0FB87F980935F0300936003109365
:101E7000610360915E0370915F03809160039091B4
:101E80006103DF91CF911F910F91FF90EF90DF9051
:101E9000CF90BF90AF909F908F900C94270EDF91C2
:101EA000CF911F910F91FF90EF90DF90CF90BF9057
:101EB000AF909F908F900895EEE5F3E02081221F70
:101EC0002227221F30915F03432F440F842F822B40
:101ED00037FB992790F90C9668E671E00E94F42D83
:101EE000438162810C94B00E20915E03221F222751
:101EF000221F30915F03432F440F842F822B37FB27
:101F0000992790F98C3091051CF4845A9E4F01C09A
:101F10000C9768E671E00E94F42D40916103609196
:101F200060030C94B00EEEE5F3E08081881F8827F3
:101F3000881F90915F03292F220F97FB992790F913
:101F400043816FEF822B0C94B00EEEE5F3E08081BD
:101F5000881F8827881F90915F03292F220F97FBE6
:101F6000992790F9438160E0822B0C94B00E409148
:101F70006103842F90E0843F910514F4445F01C015
:101F80004FEF80915E03881F8827881F90915F0321
:101F9000292F220F97FB992790F960916003822BDC
:101FA0000C94B00E40916103842F90E00C9714F0D4
:101FB0004C5001C040E080915E03881F8827881F35
:101FC00090915F03292F220F97FB992790F9609139
:101FD0006003822B0C94B00E90915E0390FF42C080
:101FE0009178811102C0926007C0833210F094642E
:101FF00003C08F73880F982B90935E0360915E03EC
:1020000070915F0380916003909161030E94270E9D
:1020100080915E03982F9E77923019F41092690296
:1020200010C0982F96959F732EE3290F2F73273199
:1020300020F491E09093690204C0995D9F739A30F7
:1020400068F3881F8827881F90915F03292F220F2C
:1020500097FB992790F94091610360916003822B6F
:102060000C94B00E089580912C03816080932C0312
:1020700081E080936A020E940D20811104C00E94B9
:10208000EC1F0E942D0E0E94230E60935E0370933E
:102090005F0380936003909361036E7761F40E9405
:1020A0002D0E0E94230E60935E0370935F03809356
:1020B00060039093610381E08093690280915E03E5
:1020C00080FF04C086958F730C94EC0F0895809167
:1020D0005E0386958F738F5F833208F081E00C94E6
:1020E000EC0F80915E03982F909590FB80F9809380
:1020F0005E0360915E0370915F0380916003909135
:1021000061030E94270E80915E0380FF04C08695C4
:102110008F730C94EC0F109269022FEF80E792E01E
:10212000215080409040E1F700C000000C94400E28
:10213000CF93C82F80916702909168020E94AE20D1
:10214000EC2FF0E0E753FB4FE491F0E08E179F0790
:1021500018F10E94A2209093680280936702E09198
:102160006602F0E0E353FB4F449180915E03881FC9
:102170008827881F90915F03292F220F97FB9927AB
:1021800090F960916003822B0E94660E8091660236
:1021900090E0019680936602CF910895CF93C82F67
:1021A00080916402909165020E94AE20EC2FF0E0D5
:1021B000EA53FB4FE491F0E08E179F07E8F00E948E
:1021C000A220909365028093640240916103609124
:1021D000600380916202909163020E94660E80917A
:1021E000620290916302019668E671E00E94E02D20
:1021F0009093630280936202CF910895CF92DF9211
:10220000FF920F931F93CF93DF93F82E809160027C
:10221000909161020E94AE20EF2DE695F0E0EA5326
:10222000FB4FE491F0E08E179F07E8F10E94A22097
:10223000909361028093600206E613E0C0E0D0E074
:1022400088E6C82EDD24D39480915E0290915F02CF
:102250008C0F9D1FB6010E94E02D980140916103F3
:10226000609160030E94AF0D68960C5F1F4FC836E7
:1022700081E0D80749F70E94400E20915E0230911C
:102280005F02F0FE0AC0C9010196BE010E94E02D66
:1022900090935F0280935E0206C021503109309313
:1022A0005F0220935E02DF91CF911F910F91FF900B
:1022B000DF90CF9008958F929F92AF92BF92CF926E
:1022C000DF92EF92FF920F931F93CF93DF93C82F6C
:1022D00080FF03C0DD24DA9402C0DD24D394809112
:1022E0005C0290915D020E94AE20C695EC2FF0E05A
:1022F000ED53FB4FE491F0E08E179F0708F467C0A1
:102300000E94A22090935D0280935C0296E6E92EE3
:1023100093E0F92E08E613E0C0E0D0E027E0822E3B
:10232000912CF80131971082F7011082F801108288
:1023300087E0A82EB12CC12C80915B028C0D87FD0B
:10234000815F082E000C990BC817D907E9F420917A
:1023500061032A9DC0012B9D900D1124B4010E94A0
:10236000F42D462F80915E03881F8827881F909147
:102370005F03592F550F97FB992790F997016091AB
:102380006003852B0E94AF0DCD0CF1E0AF1AB108B0
:1023900099F6219684E0E80EF11C0C5F1F4FCF30B8
:1023A000D10509F0BECF0E94400E80915B0291E002
:1023B000D91206C0811102C08EE007C0815005C04D
:1023C00090E00196BE010E94F42D80935B02DF91A4
:1023D000CF911F910F91FF90EF90DF90CF90BF9022
:1023E000AF909F908F9008959F92AF92BF92CF929F
:1023F000DF92EF92FF920F931F93CF93DF93CDB7AE
:10240000DEB7EC970FB6F894DEBF0FBECDBF182F26
:102410008091590290915A020E94AE20E12FF0E083
:10242000E054FB4FE491F0E08E179F0708F495C04D
:102430000E94A22090935A0280935902CE010196E5
:102440007C015E0193E0A90EB11CC12CD12C870147
:10245000F50131971082F7011082F5011082912C5D
:102460009091010180915802999E800D112487FD61
:1024700004C08F301CF08EE001C080E0082E000CFC
:10248000990BC816D906A1F480915E03881F88278E
:10249000881F90915F03592F550F97FB992790F94B
:1024A00097014091610360916003852B0E94AF0DFD
:1024B0009394F7E09F12D4CF8FEFC81AD80A94E014
:1024C000E90EF11CE4E0AE0EB11CFFE0CF16D10422
:1024D00009F0BECF28E633E099E0E92EF12C4FE079
:1024E000C42ED12CC701B6010E94F42DD901119739
:1024F000FC01EE0FFF1FEE0FFF1FE00FF11F8181A8
:102500008C93119780818C938281F9018083FFEFF6
:10251000EF1AFF0A2C5F3F4F88E1E816F10411F72C
:102520000E94400E9091010180915802913049F42F
:102530008A3F2CF489EF809358028FEF08C08150B6
:102540000AC086313CF085E18093580281E0809397
:10255000010103C08F5F80935802EC960FB6F89488
:10256000DEBF0FBECDBFDF91CF911F910F91FF90C6
:10257000EF90DF90CF90BF90AF909F900895EF9233
:10258000FF920F931F93CF93DF9380915602909108
:1025900057020E94AE20883E9340D0F10E94A220B4
:1025A0009093570280935602C0915402D0915502E5
:1025B0002196C170DD27D0935502C093540286E660
:1025C000E82E83E0F82E10E008E7812F8695FE01C3
:1025D000E80FF11DCF0181709927970140916103A8
:1025E00060916003FC010E9FC0010F9F900D1124AC
:1025F0000E94AF0D1F5FF4E0EF0EF11C1F3029F7B2
:10260000DF91CF911F910F91FF90EF900C94400EAE
:10261000DF91CF911F910F91FF90EF9008958091DE
:102620006902882391F190915E03892F86958F73BB
:102630002EE3280F2F73243018F482500C94981036
:102640002AE3280F2F73233018F486500C94CE10F1
:1026500027E3280F2F73263018F489500C94FE10AE
:1026600021E3280F2F73263018F48F500C945B1140
:102670002BE2280F2F73233018F485510C94F4119A
:102680009E77903311F40C94BF12089590937002CA
:1026900080936F020895E0916F02F091700230977D
:1026A00021F00190F081E02D099480E00895E091FF
:1026B0006F02F0917002309721F00280F381E02DDB
:1026C00009940895E0916F02F0917002309721F023
:1026D0000480F581E02D0994089520916D023091D8
:1026E0006E028217930771F090936E0280936D02D1
:1026F000E0916F02F0917002309721F00680F7812F
:10270000E02D0994089520916B0230916C0282179C
:10271000930771F090936C0280936B02E0916F02CB
:10272000F0917002309721F00084F185E02D09943A
:10273000089508950C9499130E9499200E9404050D
:102740000E9420210C943310CF92DF92EF92FF92DF
:102750000F931F93CF93DF93CDB7DEB72B970FB6B1
:10276000F894DEBF0FBECDBF0E94700582E7C82E71
:1027700082E0D82E00E010E0E02E802F0E9452066A
:10278000F60141916F01F42EF826B1F40F5F1F4F4F
:102790000E30110589F78FEF89838A831B820E948F
:1027A000A2208160782F9D838C8349815A816B811F
:1027B0008D810E94831440C090912C0391FF04C02E
:1027C0008B870E9458068B8520E030E04F2D50E02B
:1027D000922FBA01022E02C0759567950A94E2F70E
:1027E00060FF24C02E83EF8221E030E0690102C047
:1027F000CC0CDD1C9A95E2F790E08C219D21892B71
:1028000009F420E028870E94A2208160782F9A870F
:1028100089874E815F8168858A850E948314F801CB
:10282000EE58FD4F8081C826C08206C02F5F3F4F03
:102830002630310569F6AACF0E94B32210917102A9
:102840000E944B131817A1F00E944B138093710242
:102850002B960FB6F894DEBF0FBECDBFDF91CF91A0
:102860001F910F91FF90EF90DF90CF900C94A508EF
:102870002B960FB6F894DEBF0FBECDBFDF91CF9180
:102880001F910F91FF90EF90DF90CF900895DC01A2
:1028900011962C9111978C91682F70E041E050E0D7
:1028A00001C0440F8A95EAF712968C91129730E096
:1028B000882329F080918F028823E9F006C0F9016E
:1028C000E058FD4F90819423B1F086E0829FF001A3
:1028D000839FF00D1124E60FF71FEE0FFF1FEC5E34
:1028E000FE4F808191818D939C93F901E058FD4FBB
:1028F0008081482B06C0F901E058FD4F409580814A
:10290000482340830895CF93DF93CDB7DEB72B974D
:102910000FB6F894DEBF0FBECDBF942F4F83252F87
:10292000588769877A878B874A855B85452B21F095
:102930002F3F09F59F3FF9F4DE01119686E0FD0176
:1029400011928A95E9F785E0FE01379601900D9284
:102950008A95E1F749815A816B817C818D819E81C5
:102960000E94761B2B960FB6F894DEBF0FBECDBF2C
:10297000DF91CF910895CE0107960E944714DCCFD6
:10298000CF93882309F4CDC0C82F823859F40E9410
:102990004B1381FDC6C089E30E949D1E0E946D1FDE
:1029A00089E30CC0833879F40E944B1380FDB9C0D1
:1029B00083E50E949D1E0E946D1F83E50E94DF1E1D
:1029C000CF910C946D1F843859F40E944B1382FDF3
:1029D000A8C087E40E949D1E0E946D1F87E4EECF71
:1029E0008CEF8C0F813A48F48C2F0E94F3248111D4
:1029F00098C08C2F0E949D1EE3CF80E28C0F883000
:102A000048F4C77081E001C0880FCA95EAF70E94B8
:102A1000261FD6CF8BE58C0F833078F4C53A29F08A
:102A2000C63A31F083E890E005C081E890E002C04A
:102A300082E890E0CF910C946D1388E58C0F85317E
:102A400008F06FC0C83A61F1C93A69F1CA3A71F148
:102A5000CB3A79F1CC3A81F1CB3B89F1CC3B91F186
:102A6000CD3A99F1C03BA1F1CE3AA9F1CF3AB1F1FB
:102A7000C13BB9F1C23BC1F1C33BC9F1C43BD1F188
:102A8000C53BD9F1C63BE1F1C73BE9F1C83BF1F1E8
:102A9000C93BF9F1CA3B09F43FC080E090E03EC079
:102AA00082EE90E03BC089EE90E038C08AEE90E084
:102AB00035C085EB90E032C086EB90E02FC083EB11
:102AC00090E02CC084EB90E029C087EB90E026C01A
:102AD0008CEC90E023C08DEC90E020C083E891E086
:102AE0001DC08AE891E01AC082E991E017C084E92C
:102AF00091E014C081E292E011C083E292E00EC046
:102B000084E292E00BC085E292E008C086E292E0A7
:102B100005C087E292E002C08AE292E0CF910C9475
:102B20008313CF910895882309F44BC0823859F458
:102B30000E944B1381FF45C089E30E949D1E0E94A5
:102B40006D1F89E30CC0833871F40E944B1380FF22
:102B500038C083E50E949D1E0E946D1F83E50E9480
:102B6000DF1E0C946D1F843859F40E944B1382FFB2
:102B700028C087E40E949D1E0E946D1F87E4EFCF4E
:102B80009CEF980F913A58F390E2980F983050F4D8
:102B9000877091E001C0990F8A95EAF7892F0E940A
:102BA0002C1FDFCF9BE5980F933020F480E090E05E
:102BB0000C946D13885A853120F480E090E00C94D9
:102BC00083130895882321F00E94261F0C946D1F03
:102BD0000895882321F00E942C1F0C946D1F0895E6
:102BE0008F929F92AF92BF92CF92DF92EF92FF921D
:102BF0000F931F93CF93DF931F92CDB7DEB77C0166
:102C0000C72EFC01058102950F701281112321F05E
:102C100069830E94431F698169830E94961E6981AE
:102C2000882381F0112371F080E2860F883050F004
:102C300082E00E947F1E0E94961E91E0D82ED92627
:102C4000698101C0D12CAC2CA2948FE0A822B12CB8
:102C5000F501E159FF4F0C94082E8C2D807F0C2D2F
:102C60000F70882311F00295007F1123C1F000231B
:102C700009F4D2C180E2860F883010F0611105C0DE
:102C8000802F69830E94261F04C0802F69830E94C1
:102C9000361F698169830E946D1F6981BDC1862FBE
:102CA00069830E9493156981002309F40EC280E2B2
:102CB000860F883010F0611104C0802F0E942C1FF5
:102CC00003C0802F0E943C1F0E946D1FFEC19C2DDF
:102CD000907F8C2D8F70903211F08295807F6623CB
:102CE00019F06130B1F01EC0112349F0002309F43E
:102CF0004BC1013009F048C10E94561FE6C10023B4
:102D000019F0013009F4E1C189830E94591F8981BA
:102D100041C1112321F0023008F0D7C135C10111A2
:102D2000D4C138C1112321F0002309F42DC174C18D
:102D3000002309F42FC181C18C2D8695869583705F
:102D400090E0009719F0019761F0BFC1112321F0C5
:102D5000862F9C2D937002C080E090E00E946D133E
:102D6000C4C1112321F0862F9C2D937002C080E0F6
:102D700090E00E948313B9C11123F9F0653F51F02F
:102D8000663F71F0643FA9F48091A2039091A30380
:102D900081600BC08091A2039091A303826005C063
:102DA0008091A2039091A30384609093A3038093E6
:102DB000A203862F0E94BB211EC0653F51F0663FD3
:102DC00071F0643FA9F48091A2039091A3038E7FD8
:102DD0000BC08091A2039091A3038D7F05C08091C9
:102DE000A2039091A3038B7F9093A3038093A203EC
:102DF000862F0E9423220E94A82277C18C2D8370E7
:102E000009F052C011116DC1862F82958695877089
:102E1000880F880F962F9F70892E912CA12CB12C92
:102E2000082E04C0880C991CAA1CBB1C0A94D2F75B
:102E300064FF14C00FE010E020E030E0B901A80109
:102E400004C0440F551F661F771F8A95D2F7CB0128
:102E5000BA01609570958095909503C060E070E030
:102E6000CB012C2D26952695237030E0223031059C
:102E700069F02330310589F0682979298A299B294D
:102E80002130310571F00E94B91C2BC168297929C4
:102E90008A299B290E94CB1C24C10E94B91CC50110
:102EA000B4010E94A71C1DC1112319F08C2D817043
:102EB00001C08695882309F414C1862F82958695D2
:102EC0008770880F880F962F9F70892E912CA12CC8
:102ED000B12C082E04C0880C991CAA1CBB1C0A9497
:102EE000D2F764FF14C00FE010E020E030E0B90139
:102EF000A80104C0440F551F661F771F8A95D2F79B
:102F0000CB01BA01609570958095909503C060E003
:102F100070E0CB012C2D269526952370422F50E092
:102F20004230510569F04330510589F0682979290B
:102F30008A299B294130510571F00E947D1DD1C025
:102F4000682979298A299B290E948F1DCAC00E945D
:102F50007D1DC501B4010E946B1DC3C0862F90E08A
:102F6000FC01E05EF109E531F10508F051C0E158DE
:102F7000FF4F0C94082E062F0F708C2D8F7111238C
:102F800031F00E94041D802F0E94E2159EC00E9415
:102F9000251D802F0E94E91598C0112339F00111D9
:102FA00094C08C2D8F710E944A1D8FC0023008F092
:102FB0008CC0F7CF112339F08C2D8F710E94041D26
:102FC00084C01123C9F38C2D8F710E94251D7DC0F3
:102FD000112329F08C2D8F710E94EF1C76C00E9466
:102FE000EA1C73C0112351F01C2D1F71812F0E9408
:102FF000041D63E0812F0E94761E67C081E00E945D
:103000007F1E023008F461C082E00E947F1E5DC016
:10301000112331F0002381F2862F0E94C01455C085
:10302000002389F2693349F45FEF77EE83E0515072
:1030300070408040E1F700C00000862F0E94931589
:1030400044C04C2D4F70C7010E9459060E941A1CA3
:103050004CC0623F99F128F4603F49F0613FE1F0D4
:1030600020C0643FA1F050F0653F59F01AC0112311
:1030700039F190918F0281E0892706C081E01827FD
:103080001DC011111DC081E080938F0219C0111164
:1030900017C010928F0214C0002381F0111110C0CC
:1030A000E8CF002359F0862F6983112319F00E947D
:1030B000C01402C00E949315698102C010938F0250
:1030C0004C2D4F70C7010E94A70898E0A916B104C3
:1030D00041F05CF0FAE0AF1AB10822E0A216B104A8
:1030E00020F40E944B130E94A508DD20F1F00E94FD
:1030F000721E80FD1AC0F70112820E946C1E0E948F
:10310000041DC7010E94A3180E946C1E0F90DF913E
:10311000CF911F910F91FF90EF90DF90CF90BF90D4
:10312000AF909F908F900C94251D0F90DF91CF91C1
:103130001F910F91FF90EF90DF90CF90BF90AF90D5
:103140009F908F9008950F931F93CF93DF93EC017F
:10315000888199812B813C81232BB9F09F3F11F409
:103160008F3F99F0CE010E94C906882371F06881D3
:1031700079818A810E94491E8C010E94A11D0E94B2
:10318000A41CB801CE010E94F015DF91CF911F91D0
:103190000F9108950E94431F0E94531F0E94151F04
:1031A0000E946D1F0E9458230E94A82280E090E098
:1031B0000E946D1380E090E00C9483130E94331FF3
:1031C0000C94CA180E943E1EE92FE295EF70F0E0C1
:1031D0003297EE30F105B0F4EC56FF4F0C94082E08
:1031E000803F91F018F4803E68F40EC0843F51F4A3
:1031F0000BC0803E48F0813F29F406C093FB88272E
:1032000080F9089580E0089581E00895CF93DF93D9
:1032100000D000D01F92CDB7DEB70F900F900F9067
:103220000F900F90DF91CF910895CF93DF9300D04F
:1032300000D000D0CDB7DEB726960FB6F894DEBF2B
:103240000FBECDBFDF91CF9108951F93CF93DF9332
:10325000C091900216E080919102C81799F0D0E0D9
:103260001C9FF0011D9FF00D1124EE56FD4F408173
:10327000518162817381848195810E941519219603
:10328000C770E9CFDF91CF911F9108954091C2029D
:103290005091C3026091C4027091C5028091C60230
:1032A0009091C7020C9415198091C70282958F7076
:1032B00009F054C08091C402882309F44FC0809162
:1032C0009002A09191026091C2027091C30240915C
:1032D000C5025091C602B6E08A1709F43FC090E0DB
:1032E00041155105C1F17F3F11F46F3FA1F1B89F26
:1032F000F001B99FF00D1124EE56FD4F218172139C
:103300002AC02081621327C02281211124C0238179
:1033100034812417350710F421503109241B350B53
:10332000283C3105C0F42091C7022F702061209302
:10333000C70226E0289FF001299FF00D1124E956CD
:10334000FD4F80818F708061808382EC92E00E94CB
:10335000A3180C94251901968770BECF0895CF92BB
:10336000DF92EF92FF920F931F93CF93DF93CDB72E
:10337000DEB762970FB6F894DEBF0FBECDBF8C01EB
:1033800085E0F801DE011D9601900D928A95E1F726
:10339000D8014C9111965C91119712966C911297ED
:1033A0001396CD90DC9014973091C2027091C302B5
:1033B0008091C5029091C602009709F46BC17F3FCE
:1033C00019F43F3F09F466C1E090C402EE2009F40D
:1033D000C0C02091C702C816D90628F0F601E81B24
:1033E000F90BCF0104C0809590958C0D9D1DFF2495
:1033F000F394883C910578F0F12C207F09F0C6C049
:103400007C2DD98AC88A89890E94061982EC92E0AB
:103410000E94A318B1C0822F807F09F046C07513A7
:1034200014C0341312C0611110C02F70206120939A
:10343000C7020E94461982EC92E00E94A318809174
:10344000C702D80115968C932EC0CD2819F15F3F85
:1034500011F44F3FF9F0F62E61111CC080919002DB
:103460002091910236E0821709F45AC090E0389F0B
:10347000F001399FF00D1124EE56FD4F7181571365
:1034800006C07081471303C07281711103C0019699
:103490008770E9CFF62E662309F418C18091C70220
:1034A00081608093C702F12C11C1751308C03413D9
:1034B00006C0611104C08091C702D801C3C04D8706
:1034C0005E878D859E856A8B0E94E2186A898823B3
:1034D000E1F16623D1F12091C702822F82958F708E
:1034E00090E0029774F08091C2029091C302988795
:1034F0008F831986DB86CA862C87CE0107960E94A9
:10350000A31886E0F801A2ECB2E001900D928A9532
:10351000E1F70E9454190E944619FF24F394D6C083
:103520004D875E878D859E850E943E1E292F2295A0
:103530002F7030E0223031050CF0BCC09F7009F0D4
:10354000B6C0805E883008F4C1C0C8010E94A318CC
:10355000E4CFC816D90608F453C0F601E81BF90BEE
:10356000CF01883C910508F450C0F12C7C2DD98AFC
:10357000C88A89890E940619E2ECF2E086E0DF0140
:103580001D928A95E9F70E944619A0C0751314C0D0
:10359000341312C0611110C08091C702F8018583F5
:1035A000C8010E94A31886E0E2ECF2E0DF011D9260
:1035B0008A95E9F7FE2C8AC04D875E878D859E85AA
:1035C0006A8B0E94E2186A89882309F4BECF6623B9
:1035D00009F4BBCF2091C702822F82958F7090E0B3
:1035E00002970CF48ECF8091C2029091C3029A830D
:1035F00089831B82DD82CC822E83CE0101967FCF10
:10360000809590958C0D9D1DACCFF62E662309F408
:103610009CCF75132EC034132CC02091C70220FDFF
:103620001FC0822F82958F70D9F0D80115962C93E8
:1036300015978F3049F08F5F982F9295907F822F4A
:103640008F70892B15968C93C8010E94A31886E071
:10365000F801A2ECB2E001900D928A95E1F793CFC8
:1036600086E0F801A2ECB2E001900D928A95E1F7B4
:103670002DC04D875E878D859E850E94E218811141
:1036800040CF8091C70281608093C702C8010E9429
:10369000A3181CC0662309F458CF4D875E878D851B
:1036A0009E850E94E218882309F44FCF2ACF81110A
:1036B00048CF0CC0243031050CF047CF9F7009F47F
:1036C00040CFF8019581907F09F03BCF8F2D629616
:1036D0000FB6F894DEBF0FBECDBFDF91CF911F9123
:1036E0000F91FF90EF90DF90CF9008951F93CF93AD
:1036F000DF93CDB7DEB72C970FB6F894DEBF0FBEC1
:10370000CDBF4F83588769877A878B879C87CE0187
:1037100007960E94AF19882369F08F8198852A85C2
:103720003B85232BF1F19F3F09F063C08F3F09F0E8
:1037300060C037C086E0FE013796DE011196019029
:103740000D928A95E1F76F817885EA85FB85309740
:1037500041F17F3F11F46F3F21F12091910230E060
:10376000C9010196877099274091900250E0841713
:10377000950709F447C069837A83FD83EC8396E05B
:10378000929FD001939FB00D1124AE56BD4FFE0104
:10379000319601900D929A95E1F7809391020E94E3
:1037A000251916E080919002909191028917C1F13C
:1037B000189FC00111248E569D4F0E94AF19882377
:1037C00079F1E09190021E9FF0011124EE56FD4F19
:1037D0004081518162817381848195810E94151994
:1037E0008091900290E001968770992780939002D3
:1037F000D9CF4F81588569857A858B859C850E94B4
:103800001519CFCF0E94DE181092910210929002EB
:10381000E2ECF2E086E0DF011D928A95E9F7C1CF84
:103820002C960FB6F894DEBF0FBECDBFDF91CF91BF
:103830001F910895EF92FF920F931F93CF93DF9301
:103840008C01892B09F46CC0F12CEE24E394E8017F
:103850002196F8018491843740F4843008F051C0F7
:10386000813081F0823019F15BC0853709F444C0A2
:10387000A8F19CE7980F903708F052C08F770E940C
:10388000931541C00E5F1F4FFE01C49180E28C0F63
:10389000883048F4C7708E2D01C0880FCA95EAF7AA
:1038A0000E94461F14C08C2F0E94C0142DC00E5FB2
:1038B0001F4FFE01C49180E28C0F883058F4C7700E
:1038C0008E2D01C0880FCA95EAF70E944C1F0E94F6
:1038D0006D1F1AC08C2F0E94931516C00E5F1F4FCC
:1038E000FE01C491CC2381F08FE99FE00197F1F7AD
:1038F00000C00000C150F6CF0E5F1F4FFE01F490D4
:1039000003C00E94C0148E018F2D882309F49FCF1D
:10391000EFE9FFE03197F1F700C000008150F5CFEB
:10392000DF91CF911F910F91FF90EF90089508952F
:103930000E94971C60930303709304038093050314
:10394000909306030C94CA1808950C94981C0F9336
:103950001F930091030310910403209105033091FC
:103960000603602B712B822B932B1F910F910C94CC
:10397000981C0F931F93009103031091040320914F
:1039800005033091060360237123822393231F9143
:103990000F910C94981C0F931F93009103031091A7
:1039A00004032091050330910603602771278227C5
:1039B00093271F910F910C94981C08950E94DD1C71
:1039C0006093FF02709300038093010390930203BE
:1039D0000C94CA1860E070E0CB010C94DE1C0F93CD
:1039E0001F9341E050E060E070E08A019B0104C059
:1039F000000F111F221F331F8A95D2F7C901B8018A
:103A00001F910F910C94DE1C0F931F9341E050E027
:103A100060E070E004C0440F551F661F771F8A9551
:103A2000D2F78091FF0290910003A0910103B09121
:103A300002038A019B01082B192B2A2B3B2BC9015E
:103A4000B8011F910F910C94DE1C0F931F9341E05E
:103A500050E060E070E004C0440F551F661F771F00
:103A60008A95D2F740955095609570958091FF02A8
:103A700090910003A0910103B09102038A019B0180
:103A8000082319232A233B23C901B8011F910F9151
:103A90000C94DE1C0F931F9341E050E060E070E057
:103AA00004C0440F551F661F771F8A95D2F7809177
:103AB000FF0290910003A0910103B09102038A01DB
:103AC0009B01082719272A273B27C901B8011F9105
:103AD0000F910C94DE1C0F931F930091FF02109125
:103AE00000032091010330910203602B712B822B84
:103AF000932B1F910F910C94DE1C0F931F93009139
:103B0000FF02109100032091010330910203602312
:103B10007123822393231F910F910C94DE1C0F932A
:103B20001F930091FF021091000320910103309137
:103B3000020360277127822793271F910F910C940E
:103B4000DE1C0895292F220F920F990F890FA82F9D
:103B5000A695A695A695877051E001C0550F8A9548
:103B6000EAF785E0A89FD001112420E030E070E062
:103B7000F901EA0FFB1FE853FD4F4081CB01022EF4
:103B800002C0969587950A94E2F7817099278195EE
:103B900084278523842780832F5F3F4F253031057D
:103BA00039F70895292F220F920F990F890F682F47
:103BB000669566956695982F977085E0689FB00129
:103BC000112440E050E080E0FA01E60FF71FE853CF
:103BD000FD4F208130E0092E02C0369527950A94CA
:103BE000E2F721703327042E01C0220F0A94EAF76E
:103BF000822B4F5F5F4F4530510531F70895CF92CB
:103C0000DF92EF92FF920F931F93CF93DF938C017C
:103C1000C0900303D0900403E0900503F0900603E6
:103C20008091FF0290910003A0910103B0910203E3
:103C3000C82AD92AEA2AFB2ACFE1D0E0D701C60157
:103C40000C2E04C0B695A795979587950A94D2F740
:103C500080FF06C0B8018C2F0E94C208019721F492
:103C6000219760F780E001C08C2FDF91CF911F91E9
:103C70000F91FF90EF90DF90CF900895CF93DF9357
:103C8000EC010E94FF1DBE010E94C208DF91CF918E
:103C900008951F93CF93DF93EB0190918E029923A8
:103CA00021F0CB010E943E1E13C0882349F0CB01B6
:103CB0000E94FF1D182F682FCE010E94A21D04C074
:103CC000CB010E94D21D182FBE01812F0E94C20875
:103CD000DF91CF911F910895809107038595859578
:103CE00085950895809107038770089598E0899FCE
:103CF00090011124262B209307030C94041D20917E
:103D000007038095822380930703982F977069F4A7
:103D100030E0482F082E000C550B2417350729F0EA
:103D20008595859585950C94251D0895909107039B
:103D3000977081E009F480E0089590911301992330
:103D400021F09091A80397FD09C0209102013091C4
:103D50000301F90132969FEF40E01FC0982F96951E
:103D6000969596959F3150F5E0910201F0910301EF
:103D7000E90FF11D877021E030E0A90102C0440F76
:103D8000551F8A95E2F7CA019181892B8183089595
:103D90009F3F39F04F5F4E3141F051915813F8CFAA
:103DA0000DC05111F7CF942FF5CF9F3F39F0F90196
:103DB000E90FF11D97FDFA9582830895089590917A
:103DC0001301992321F09091A80397FD09C0209138
:103DD000020130910301F9013296205E3F4F1FC06E
:103DE000982F9695969596959F31F0F4E091020163
:103DF000F0910301E90FF11D877021E030E0A90186
:103E000002C0440F551F8A95E2F7CA01809591813F
:103E10008923818308953196E217F30729F0908171
:103E20009813F9CF1082F7CF089581E090E0E091E8
:103E30000201F0910301E80FF91F10820196803210
:103E40009105A9F7089580912B03089590912B0374
:103E5000892B80932B030895809590912B038923C0
:103E600080932B03089510922B03089590912A03B9
:103E7000892B80932A030895809590912A038923A2
